S018000064656D6F70726F675F786D63343730302E737265633D
S3150C0080004088FE1F058200089D8200089D8200089C
S3150C0080109D8200089D8200089D82000800000000D9
S3150C0080200000000000000000000000009D82000817
S3150C0080309D820008000000009D82000845B10008E2
S3150C0080409D8200089D8200089D8200089D82000882
S3150C0080509D8200089D8200089D8200089D82000872
S3150C0080609D820008000000000000000000000000D7
S3150C0080709D820008000000009D8200089D82000879
S3150C0080809D8200089D8200089D8200089D82000842
S3150C0080909D8200089D8200089D8200089D82000832
S3150C0080A09D8200089D8200089D8200089D82000822
S3150C0080B09D8200089D8200089D8200089D82000812
S3150C0080C09D8200089D8200089D8200089D82000802
S3150C0080D09D8200089D8200089D8200089D820008F2
S3150C0080E09D8200089D8200089D8200089D820008E2
S3150C0080F09D8200089D8200089D8200089D820008D2
S3150C0081009D8200089D8200089D8200089D820008C1
S3150C0081109D8200089D8200089D8200089D820008B1
S3150C0081209D8200089D8200089D8200089D820008A1
S3150C0081309D8200089D8200089D8200089D82000891
S3150C0081409D8200089D8200089D8200089D82000881
S3150C0081509D8200089D8200089D8200089D82000871
S3150C00816000000000000000000000000000000000FD
S3150C0081709D8200089D8200089D8200089D82000851
S3150C0081809D8200089D8200089D8200089D82000841
S3150C0081909D8200089D8200089D8200089D82000831
S3150C0081A09D8200089D8200089D8200089D82000821
S3150C0081B09D8200089D8200089D8200089D82000811
S3150C0081C09D8200089D8200089D8200089D82000801
S3150C0081D09D8200089D8200089D8200080000000018
S3150C0081E09D8200089D8200089D8200089D820008E1
S3150C0081F09D820008000000009D820008000000001F
S3150C008200EE11AA55DFF874D01D4880471D4C1E4D43
S3150C008210AC4209DA21686268A368043BA2BFC8585D
S3150C008220D050FAE70C34F3E7184B194CA34208DA92
S3150C00823019685A680020043AA4BF8850FBE7083333
S3150C008240F4E71448804714488047000000B2000C3D
S3150C0082504088FE1F3000000000B2000C4088FE1F54
S3150C008260000000007088FE1F1408000000000020AB
S3150C0082700000000000000020A03000004088FE1F17
S3150C008280259D00084C820008648200086482000860
S3150C0082907C82000855B1000825AE0008FEE70000F8
S3150C0082A010B4013A0A440BE00C784B7803EB042328
S3150C0082B09BB2184480B2984201D2013080B202318E
S3150C0082C09142F1D307D10B781B02184480B2984225
S3150C0082D001D2013080B25DF8044B704770B4C5789A
S3150C0082E00D44EDB2134CE57083780E0A3344DBB2C1
S3150C0082F0A37042786270007820709CB2A64206D9B0
S3150C0083000132D2B20B4C62700AB901302070C9B27C
S3150C0083108D420CDA0133DBB2064A93703BB95378C3
S3150C0083200133DBB2537013B913780133137070BC7D
S3150C008330704700BFBC89FE1F10B50146074C20686C
S3150C0083400830FFF7CBFF2368054A1178197251786C
S3150C008350597291789972D278DA7210BDCC89FE1F57
S3150C008360BC89FE1F00221A4B1A7006E00021194A1E
S3150C00837022F813100133164A1370154B1B78002B79
S3150C008380F4D00022124B1A7009E0C3EB031149001A
S3150C008390114A0A440021517001330D4A13700C4BDB
S3150C0083A01B78002BF1D04FF480620C4B1A80002204
S3150C0083B0074B1A7007E00A4A02EB831200219180E0
S3150C0083C00133034A1370024B1B78002BF3D0704712
S3150C0083D08488FE1FF089FE1FE889FE1F7888FE1F21
S3150C0083E04490FE1F00220A4B1A700BE01946094AEC
S3150C0083F032F813201AB9074B23F8110070470133D2
S3150C008400034A1370024B1B78002BEFD0704700BF4A
S3150C0084108488FE1FF089FE1F030A43EA002080B2FF
S3150C008420704700BF08B5002005491422FFF738FF36
S3150C00843010B1FFF7F1FF08BD4FF6FF7008BD00BF86
S3150C0084400E8AFE1F38B50D4D2C7C6B7C03EB042479
S3150C008450143CA4B2204480B205F11A010822FFF79D
S3150C0084601FFF05F122012246FFF71AFF10B1FFF795
S3150C008470D3FF38BD4FF6FF7038BD00BF008AFE1F14
S3150C00848008B50620FFF7DEFF08BD00BF70B5A54B8B
S3150C0084901C68042800F07181A34BA44A1360A44AFB
S3150C0084A01360032810D1637E03F00F03032B40F0F7
S3150C0084B0DA85238A002B40F0D68508229D4B1A704C
S3150C0084C002F0FEFC00F094BC02287BD19A4AD378C9
S3150C0084D00133DBB2D37063B993780133DBB293709B
S3150C0084E03BB953780133DBB2537013B913780133AC
S3150C0084F013700023914A1380914A1380637E072BD5
S3150C00850001D0052B0AD1A37E0133DBB2A376782BDF
S3150C00851040F0A9850023637600F0A5BD002B00F082
S3150C008520A285228A002A41D0A27E511EA176002A5B
S3150C00853040F09985E27E082A05D0591EC9B2012958
S3150C0085400ED8052A0CD1002363768022794B1A703B
S3150C00855002F0B6FC14227B4B83F82F2000F014BDDE
S3150C008560042A03D803219140C9B200E03021A17638
S3150C0085700132E27603F00F03013B072B00F2738501
S3150C008580DFE813F0780208000D00F2037105F20320
S3150C0085907105F20300226B4B83F82F206EE2042246
S3150C0085A0644B1A7002F08CFC00F057BC03F00F03FE
S3150C0085B0032B40F0588508225E4B1A7002F080FCA3
S3150C0085C000F016BC052817D15F4B1B689B88002B47
S3150C0085D000F049850023534A13605C4A53490A60EC
S3150C0085E053490A60564A1380544A13800822514B49
S3150C0085F01A7001F04DFAC0E0524B9B7B452B40F0B4
S3150C0086003285504A157C537C03EB05214B4A128864
S3150C008610914200F328858DB2484B1D80494B1B7D3A
S3150C00862013F03F0F40F01F85464B5B7D002B40F04F
S3150C0086301A85474B1C880CB95B885BB1414BDB8BAD
S3150C0086409C4240F010853F4B1A8C414B5B889A42FA
S3150C00865040F00985FFF7E6FE4FF6FF73984240F0AF
S3150C0086600285384BDB7D062B00F0B880112B23D00E
S3150C008670012B40F0F884334B93F82230082B40F052
S3150C008680F284304B002283F822209B8C4FF6F67234
S3150C008690934203D909332B4A938402E00833294ABF
S3150C0086A09384284B5A8BDA839A8B1A845C83284AD8
S3150C0086B052889A8300F0D3BC1C3D204B1D80254A62
S3150C0086C0214B1A6026E09A880AB31E49898C8A4285
S3150C0086D01DD1DA8832B11B49498C8A4202D0B2F5D7
S3150C0086E08A4F14D11A8812B95988002936D04FF6F8
S3150C0086F0FF718A4202D1588888422FD01149498B82
S3150C0087008A4204D10F4A918B5A88914226D0403323
S3150C0087100D4A13600C4B1B680F4A9342D3D300F0DF
S3150C008720A2BC00BFCC89FE1F368AFE1FC889FE1F5D
S3150C008730B889FE1FC089FE1F7488FE1FB489FE1FF0
S3150C0087404290FE1F008AFE1FC489FE1F2A8AFE1F46
S3150C008750FC89FE1F4490FE1F8490FE1F0023AD4A29
S3150C00876013600221AC4A1170AC4AAD490A60AD499E
S3150C0087700A60AD4A138001F08BF9AB4B1A88002ABC
S3150C00878000F0718402F11C0189B2A84B1980A84B28
S3150C008790080A18745974A7490968087A987511203B
S3150C0087A0D875083292B2100A40EA0222DA84002204
S3150C0087B083F8282083F829208A885A84CA889A84C0
S3150C0087C09D4A1088588352889A830A88DA834A8885
S3150C0087D01A843633924A136000F02CBCFFF750FE15
S3150C0087E04FF6FF73984240F03E84944C17E0617E3E
S3150C0087F0A1B18F4B9A8CA3889A420FD18C4B5A8C71
S3150C008800E3889A420AD18A4B5A8B23889A4205D11D
S3150C008810874B9A8B63889A4200F04A811E34874BA9
S3150C0088209C42E4D9824B93F82F3003F03F03022B82
S3150C00883014D17F4B9B8C99B2814A13800022814BB9
S3150C0088401A7007E0804A32F8132091425BD001334C
S3150C0088507C4A13707B4B1B78002BF3D0744B93F82C
S3150C0088602F3013F0040F40F0FE83714B142283F863
S3150C0088702F2028216D4A1180502283F82E2093F840
S3150C008880290093F82D2083F8292093F8281093F8C3
S3150C0088902C2083F8282083F82C1093F8272093F8A3
S3150C0088A02B4083F8274083F82B2093F82640654D00
S3150C0088B02C7093F82A5083F8265083F82A400130FE
S3150C0088C0C0B283F82D0068B94B1CDBB2584981F84D
S3150C0088D02C303BB9531CDBB281F82B3013B9013465
S3150C0088E081F82A40524B5A8C55490A80998C5984E6
S3150C0088F09A845A8BDA839A8B1A844F4A1188598335
S3150C00890052889A8381E300244E4B1C701CE0194656
S3150C0089101E224A4802FB0302527E1AB91E2404FB8D
S3150C008920010415E0072A0CD13CB11E22434902FB77
S3150C0089300312917EA27E914203D9404A1E2404FB67
S3150C008940032401333F4A13703E4B1B78002BDED0B9
S3150C008950002C00F088832F4B1C600323A376237610
S3150C0089600023A3750422E275E376314DAB8CA3800C
S3150C0089706B8CE3806B8B2380AB8B638001206076E2
S3150C008980324B1A7822735A7862739A78A273DB7810
S3150C008990E373208295F82930E37295F82830A37298
S3150C0089A095F82730637295F826302372FFF7C4FCCE
S3150C0089B095F82E0000F0F003502B5BDD0022214BC6
S3150C0089C01A704FE003F13602194DAA5C204D2A703D
S3150C0089D0002A4FD0012A03D101331A4A137041E001
S3150C0089E0022A37D103F13702114DAA5C042A31D180
S3150C0089F001F13803EA5C39316B5C43EA0222104B15
S3150C008A001A8040F20A63934228BF13466382A382FC
S3150C008A1030E000BFCC89FE1FC089FE1F2A8AFE1FCC
S3150C008A20C889FE1FB889FE1F4290FE1FB489FE1F1F
S3150C008A30008AFE1FC489FE1FFC89FE1FD089FE1FFB
S3150C008A407088FE1F8488FE1FF089FE1F7488FE1F27
S3150C008A508588FE1F03F13702A7498A5C52B113447D
S3150C008A60A64A1370A54B1B7819460209053AB3EBB7
S3150C008A70820FA7DB1022A04B83F82F209E4B93F876
S3150C008A802F2042F0020283F82F20022283F8362090
S3150C008A90042283F83720062283F838200A2283F82A
S3150C008AA039202C21964A1180602283F82E2072E2FE
S3150C008AB0944B1C600022944B1A708F4B93F82F200A
S3150C008AC012F0040F07D00023637620228E4B1A7007
S3150C008AD002F0F6F9C7E2884B93F82E301B099B007F
S3150C008AE086480370EB1A143B9BB28548038001F051
S3150C008AF00F01022903D102F03F0112290FD013B93D
S3150C008B0012F0030F0BD07C4BD98C2389994240F081
S3150C008B103782794B198D6389994240F0318212F074
S3150C008B20100F48D0218A002945D004F10C00FFF71C
S3150C008B30D5FB714B93F82A30744A107883423AD19C
S3150C008B406D4B93F82B3051788B4234D16A4B93F89A
S3150C008B502C30927893422ED1674B93F82D506B4B59
S3150C008B60DB789D4227D120736173A273E373E37E96
S3150C008B70D3B9237EA27E9A1AA17DA2EBD10202F072
S3150C008B80FF02D3B21144C9B2A17513F0800F01D004
S3150C008B905242D3B2E07DA3EB900250FA82F2D3B2EA
S3150C008BA0E37503EBD10323760122574B1A70237E10
S3150C008BB0A37600232382617E01F00F03013B072B72
S3150C008BC000F25182DFE813F008002300AA007601B8
S3150C008BD0A601C201DC0168014B4B1B7813F0010F97
S3150C008BE000F04182032363764022474B1A70002320
S3150C008BF02382434B188820B14222434B1A70FFF74D
S3150C008C009BFB0022424B1A8002F05AF9F0E03E4BD5
S3150C008C101B7813F0010F65D0374B93F82F3003F008
S3150C008C203F03122B5ED1344B93F82E0000F0F00369
S3150C008C30502B39DD0022314B1A702DE003F1360230
S3150C008C402D4DAA5C334D2A7072B3012A03D1013320
S3150C008C502A4A137020E0022A16D103F13702264D58
S3150C008C60AA5C042A10D101F13803EA5C39316B5C39
S3150C008C7043EA0222284B1A8040F20A63934228BF29
S3150C008C8013466382A3820FE003F137021A498A5C0A
S3150C008C9052B11344194A1370184B1B781946020922
S3150C008CA0053AB3EB820FC9DB03236376124B93F8B9
S3150C008CB02620227293F82720627293F82820A2723B
S3150C008CC093F82930E3720120FFF736FB42220E4B54
S3150C008CD01A70002323820A4A13800D4A138002F06D
S3150C008CE0EFF885E02022084B1A7002F0E9F8054BE4
S3150C008CF01B6800225A76B1E5008AFE1F8488FE1F87
S3150C008D00B489FE1FCC89FE1FC089FE1FBC89FE1FBD
S3150C008D104290FE1F8588FE1F7088FE1F914B93F8AC
S3150C008D202F3013F0010F24D011F0100F21D1238A0C
S3150C008D30002B40F098818C4D2888013080B2FFF7CB
S3150C008D40FBFA8A4A137843F0100313702A881AB177
S3150C008D5043F00203854A137002F0B2F80123238212
S3150C008D60082363760023E37611227E4B83F82F20AB
S3150C008D700AE113F0200F10D07A4890F834301A021A
S3150C008D8090F8353042EA0300794D2E68304428605D
S3150C008D90754813430288D31A0380734B188848B15D
S3150C008DA011F0100F06D1714A137843F002031370B9
S3150C008DB0FFF7C2FA6B4A92F8301092F8313003EB97
S3150C008DC001239BB26B4A1380A28A934200D80BB93B
S3150C008DD0684B1A80674B1B886382644B1B7813F0B5
S3150C008DE0030F00F040810022634B1A8002F068F8F2
S3150C008DF05E4B1B7813F0200F08D000235E4A1380BD
S3150C008E0063761422574B83F82F20BDE013F0100F16
S3150C008E100CD00023584A1380012222820422627647
S3150C008E20E37611224F4B83F82F20ADE0524A12887D
S3150C008E308AB113F0010F01D000232382238A43B990
S3150C008E40638A9A4201D94C4A13804B4B1B88238266
S3150C008E5001E0494A13800023E376484B1A68444BD9
S3150C008E601A60454B1B884BB1238A3BB128333E4ACB
S3150C008E70138018223B4B83F82F2088E03B4B1B7842
S3150C008E8013F0020F00F0EF802822374B1A801022C5
S3150C008E90344B83F82F207AE0344B1B7813F0010FF8
S3150C008EA000F0E180002363761022304B1A7002F03A
S3150C008EB007F8D8E02C4B188808B1FFF73DFA294B78
S3150C008EC093F82F3013F0010F15D0284B1B7813F0A5
S3150C008ED0010F05D0072363760023A376238201E0D6
S3150C008EE0062363760120FFF727FA10221F4B1A7010
S3150C008EF001F0E6FF44E01D4B1B7813F0010F04D084
S3150C008F000523637600232382ADE0174B1B88002BC9
S3150C008F1036D1A8E0144B188808B1FFF70DFA114B9F
S3150C008F2093F82F3013F0010F0CD007236376002330
S3150C008F30A3760120FFF700FA10220C4B1A7001F0F1
S3150C008F40BFFF1DE0084B1B88D3B98CE0074B1B7881
S3150C008F5013F0010F00F08780072363760023A376B6
S3150C008F6081E000BF008AFE1FB489FE1FC089FE1F68
S3150C008F70C889FE1F7088FE1F4290FE1FB889FE1F0F
S3150C008F8010223C4B83F82F2028223B4B1A80502270
S3150C008F90384B83F82E20227A364B83F82A20627AB5
S3150C008FA083F82B20A27A83F82C20E27A83F82D20E2
S3150C008FB0227B83F82620627B83F82720A27B83F80A
S3150C008FC02820E27B83F829200622DA75A2885A84A7
S3150C008FD0E2889A84294A1188598352889A8322886E
S3150C008FE0DA8362881A84637E13F0100F06D0214B45
S3150C008FF0002283F8312083F8302006E01D4B062230
S3150C00900083F830200A2283F831201A4C4023A375AA
S3150C009010194B1B881A0A22746374002384F83530A2
S3150C00902084F8343084F8323084F83330FFF728FA79
S3150C009030C04360860F4C4523A3730022E27362750E
S3150C00904022750F490B8801339BB20B80190AA17448
S3150C009050E37422766276FFF7E5F9C043208300229B
S3150C009060084B1A7070BD0023034A1380054A13700F
S3150C00907070BD00BF008AFE1FB489FE1FFC89FE1F4F
S3150C0090807288FE1FC089FE1FF8B505460E46284A93
S3150C009090138801339BB21380B3F5FA4F03D34FF405
S3150C0090A08052234B1A800022224B1A700CE0224B62
S3150C0090B003EB84139F881E4B1888FFF7ADF9874284
S3150C0090C0E5D001341B4B1C701A4B1C78002CEED0CF
S3150C0090D000221A700BE0184A02EB831292881AB916
S3150C0090E0154800EB831007E00133124A1370114B3D
S3150C0090F01B78002BEFD00020C0B10D4B1A88130A39
S3150C00910043EA02238380C6804DB90346002203F846
S3150C009110012B4270013303F8012B1A7003E02B88E4
S3150C00912003806B88438040230372F8BD0020F8BD92
S3150C0091307888FE1F8488FE1F4490FE1F00290CDDD4
S3150C00914008B503468AB205490A8005490868834270
S3150C00915002D0194602F034F808BD70474290FE1F43
S3150C009160B889FE1FF0B400223B4B1A703B4D1EE033
S3150C0091703A4C5A001A449200A518A45AA4B103EB0F
S3150C00918043029200354F3A4452886AB10788BC4272
S3150C0091900AD14488A24207D10C686C60898829815F
S3150C0091A02F4B1B78AB7254E001332B4A13702A4BAE
S3150C0091B01B78072BDCD90022274B1A700FE0274CA3
S3150C0091C05A001A449200A518A25A2AB903EB430274
S3150C0091D092002244528832B101331F4A13701E4B3F
S3150C0091E01B78072BEBD9082B28D100231D4A1370AB
S3150C0091F01D4A1370184A137013E0194A157803EBBD
S3150C0092004304A400194A22449278AE1A154C2478C9
S3150C009210A64203DD134A1670134A137001330E4A25
S3150C00922013700D4B1B78072BE7D90F4B1D780A4B88
S3150C0092301D7005EB45039B00084D1D4402682B462B
S3150C00924043F8042B0A686A608A889A80044B1B7858
S3150C009250AB72F0BC704700BF8688FE1F8888FE1F65
S3150C009260E988FE1F8788FE1FE888FE1F9088FE1F70
S3150C00927070B4174B18780130C0B218700022154B19
S3150C0092801A701EE014495A001A4492008C18895A16
S3150C00929062880A4312D003EB430189000F4A0A4441
S3150C0092A09278821A772A09DD0B4E0C467518002126
S3150C0092B031556970AA1C02F8011B11700133054A5D
S3150C0092C01370044B1B78072BDCD970BC704700BF9E
S3150C0092D0E988FE1F8688FE1F8888FE1F9088FE1F61
S3150C0092E038B5354B1B88292B03D80022324B1A80F4
S3150C0092F038BD0022304B1A80304B9B8AB3F5807FE9
S3150C00930003D0B3F5007F44D038BD2C4BDA8C2C4BF4
S3150C0093101B889A424ED1294B1A8D294B5B889A424F
S3150C00932048D1284CA51F20462946FFF71BFFA4F160
S3150C0093301C03002204F8082C022204F8072C54F80B
S3150C009340061C616034F8021C21811F49086844F828
S3150C009350060C898824F8021C44F8160C24F8121CF6
S3150C009360616844F81C1C228924F8182C9A8B62819B
S3150C0093706288A281124A11889983528862800822D7
S3150C00938004F8102C062204F80F2C2A220A4B1A80F9
S3150C00939038BD0A4BDA8C0A4B1B889A420AD1074B0A
S3150C0093A01A8D074B5B889A4204D106490846063942
S3150C0093B0FFF7D8FE38BD00BFB489FE1F008AFE1F1A
S3150C0093C0FC89FE1F1C8AFE1F7C88FE1F10B5514BA4
S3150C0093D0D98B8AB24FF6FF739A420CD14D4B188C2F
S3150C0093E04FF6FF73984206D14A4B4B4A10681860E9
S3150C0093F092889A807EE0494B1B88494800885340E6
S3150C009400184209D1434B1A8C94B2444B5B8844489E
S3150C00941040886340184206D0424B434A1188198053
S3150C00942052885A8002E03F4B19805A8000223F4BEB
S3150C0094301A703F4C16E03E495A001A4492008C189A
S3150C009440384800888A5A904209D1364A518803EB2B
S3150C00945043029200364802445288914206D00133A8
S3150C009460324A1370314B1B78072BE4D9082B3BD1AE
S3150C009470284C2046FF21062201F0ADFE002384F87D
S3150C009480203084F8213084F8223084F8233084F894
S3150C009490243084F82530274A1168C4F806109288BF
S3150C0094A06281C4F8161062831E4A1188E1845288C0
S3150C0094B022851A4A1188A1835288E28323750122D8
S3150C0094C06275A373E2730822227463740623A37471
S3150C0094D00423E3742273062363733634164B1C6021
S3150C0094E02A22164B1A8010BD0A4B54F8042F1A6008
S3150C0094F0A2889A80074B0F4A1168C3F80610928807
S3150C0095005A8108221A7300225A730C4A13880E3396
S3150C009510138010BD008AFE1FE8B10008FC89FE1FEF
S3150C009520F889FE1FEC88FE1FF489FE1F8688FE1F35
S3150C0095308888FE1F7C88FE1FC889FE1FB489FE1F03
S3150C00954010B50446416000F0FBFB206010BD00BF67
S3150C00955010B5044600F0F4FB2368C01A6368984201
S3150C009560B4BF0020012010BD3523037001234370C6
S3150C00957081700330704700BF034636220270042206
S3150C0095804270034A1068C3F80200981D704700BF6A
S3150C0095900C89FE1F3723037003234370012282704C
S3150C0095A0C370062303710530704700BFFF23037099
S3150C0095B001307047074B828C1A80C28C5A80064B3E
S3150C0095C0028D1A80428D5A80044B028E1A80428E6E
S3150C0095D05A807047FC89FE1FF889FE1FF489FE1F0E
S3150C0095E003463222027004224270034A1068C3F802
S3150C0095F00200981D704700BF1489FE1F10B4034665
S3150C009600014400242EE01A78332A24D006D8032AE3
S3150C00961010D0062A13D0012A21D106E0362A15D0FD
S3150C009620FF2A21D0352A1AD10EE0D3F80200104AAF
S3150C009630906214E0D3F802000D4A10630FE0D3F8E1
S3150C00964002000B4AD0620AE09C7808E0D3F80200CC
S3150C009650074AD06103E0D3F80200054A10625A7833
S3150C009660023213448B42CED320465DF8044B70472E
S3150C009670F088FE1FF8B504460123037043701C4B9B
S3150C0096809A6982700025C5701A4A10686060258137
S3150C00969080276781184A1268E26025746574A57480
S3150C0096A0E57425756575A575E57525766576A576D6
S3150C0096B0E5769E6904F11C005969324601F080FD7D
S3150C0096C0A0191C302946C6F1100201F084FD04F1E4
S3150C0096D02C002946402201F07EFD04F16C0029463F
S3150C0096E03A4601F078FD054B1868C4F8EC00F8BD55
S3150C0096F0F088FE1FF0B10008FC89FE1FF4B10008CB
S3150C00970038B50A4C25682846FFF7B4FF05F1F0007A
S3150C0097100121FFF729FFFFF73DFFFFF747FF2368FE
S3150C009720C11A1846FFF70AFD38BD00BFC889FE1FCF
S3150C00973038B50B4C25682846FFF79CFF05F1F00061
S3150C0097400321FFF711FFFFF717FFFFF749FFFFF79D
S3150C0097502DFF2368C11A1846FFF7F0FC38BD00BF71
S3150C009760C889FE1F10B5114B1C682378022B17D124
S3150C009770201D0F49042201F013FD98B90D4B04F17D
S3150C0097801C0059699A6901F00BFD68B92069094BEF
S3150C009790586204F1F000084B1988FFF72FFF10BD33
S3150C0097A0002010BD002010BD002010BDC889FE1F72
S3150C0097B0F0B10008F088FE1FB489FE1F10B582B008
S3150C0097C00C4C6061A1610023A3704FF6FF73ADF8DA
S3150C0097D00430ADF8063001A84FF48641FFF754FC6F
S3150C0097E0606010B14FF4884383800022014B1A80CD
S3150C0097F002B010BDF088FE1F024B00221A805A8060
S3150C009800704700BFFC89FE1F38B59E4B1B88B3F50D
S3150C009810937F7FD010D840F20F12934234D0B3F519
S3150C009820887F01D2EBB118E1B3F5887F34D040F2D2
S3150C0098302512934266D010E1B3F5AB7F00F0BF80E2
S3150C00984005D840F25512934200F0B28005E1B3F50B
S3150C009850B57F00F0CE8040F26B12934200F0D080C0
S3150C009860FBE0884B01229A704FF47A721A61FFF76B
S3150C00987047FF844C04F108002169FFF761FE40F2B2
S3150C0098800F132380002300E00123002B00F0EA8055
S3150C0098904FF488727B4B1A807B4B1B7813F0020FAC
S3150C0098A005D17A48FFF754FE002800F0DD80764B90
S3150C0098B01B7813F0020F07D0FFF754FF022803D1D1
S3150C0098C00222704B9A700CE06E4B1B694EF65F22AF
S3150C0098D0934202DC5B006B4A13616A4B9B78022B4A
S3150C0098E0C5D14FF47A72674B1A61FFF721FF654CAD
S3150C0098F004F108002169FFF723FE40F225132380AB
S3150C009900002300E00123002B00F0B0804FF493728B
S3150C0099105C4B1A805C4B1B7813F0020F05D15B482D
S3150C009920FFF716FE002800F0A380574B1B7813F0A8
S3150C009930020F07D0FFF716FF052803D10322514B60
S3150C0099409A7011E04F4B1B6942F21072934207DC7E
S3150C0099504C4A03F57A7313619378032BC5D103E054
S3150C0099600020484B188038BD4648FFF723FE454D6E
S3150C009970288CFEF751FD0404688CFEF74DFD204340
S3150C00998040084FF47A7303FB00F0002801DB2861D2
S3150C00999003E06FF000423B4B1A613A4C04F10800AD
S3150C0099A02169FFF7CDFD40F255132380002300E01B
S3150C0099B00123002B5ED04FF4AB72324B1A80334826
S3150C0099C0FFF7C6FD002857D02E4B02229A704FF493
S3150C0099D07A721A61FFF710FFFFF7AAFE294C04F101
S3150C0099E008002169FFF7ACFD4FF4B5732380002303
S3150C0099F000E00123002B41D040F26B12214B1A8060
S3150C009A00214B1B7813F0020F04D12048FFF7A0FD61
S3150C009A10002835D01C4B1B7813F0020F07D0FFF72C
S3150C009A20A1FE052803D10322164B9A7011E0154BA3
S3150C009A301B6942F21072934207DC124A03F57A73E1
S3150C009A4013619378032BC7D103E000200D4B1880CC
S3150C009A5038BD0C48FFF7AEFD89E70022094B1A808A
S3150C009A60022038BD032038BD002038BD032038BD88
S3150C009A70002038BD032038BD002038BD032038BD7A
S3150C009A80002038BDF088FE1FC089FE1FF888FE1F17
S3150C009A9008B5FFF7B9FE08BD82B00023019303E0B9
S3150C009AA000BF019B01330193019B8342F8D302B0A3
S3150C009AB0704700BF72B60D4B0D4A9A60BFF34F8FBD
S3150C009AC062B6D3F8882042F47002C3F888205A692B
S3150C009AD022F008025A61074941F214028B5823F00E
S3150C009AE00F0343F004038B50704700BF00ED00E0FA
S3150C009AF0008000080010005800487047001BB70093
S3150C009B0010B51E4BDB6813F4803F27D01C4BDB686B
S3150C009B1013F0010F02D1FFF7EFFF00E01948184BC5
S3150C009B201B6813F0040F11D015498A68C2F303623F
S3150C009B308B68C3F306238C68C4F30644611C02FBD2
S3150C009B400112B0FBF2F203FB022208E00C4B9B68FD
S3150C009B5003F07F030133B0FBF3F200E0094A074937
S3150C009B60C868C0B20130B2FBF0F3086900F001001E
S3150C009B700130B3FBF0F0044B186010BD00460050EA
S3150C009B801047005000366E01C0FF032070B5574BCE
S3150C009B901B6813F0010F09D1544A536843F00103B3
S3150C009BA05360524B1B6813F0010FFAD0504B1B68D5
S3150C009BB013F4007F08D04E4A936843F40073936005
S3150C009BC041F64C50FFF768FF4A4C636843F4002398
S3150C009BD0636040F6C410FFF75FFF636823F48033BD
S3150C009BE023F002036360444B5B6813F0300F21D003
S3150C009BF0103C636823F4702323F030036360FFF793
S3150C009C007BFF3E4BA3FB00231B0D013B626842EA24
S3150C009C1003436360374BDA6822F00102DA605A6854
S3150C009C2022F400325A60334B1B6803F46073B3F5AD
S3150C009C30607FF8D12F4B5A6842F001025A605A687D
S3150C009C4042F010025A602E4A9A605A6842F040025C
S3150C009C505A605A6822F010025A605A6842F48022FE
S3150C009C605A60244B1B6813F0040FFAD0214A536830
S3150C009C7023F0010353601F4B1B6813F0010FFAD13D
S3150C009C80204C4FF00113E3600026666126612662C4
S3150C009C9066620323E3611C4BA3611C4BA362154D47
S3150C009CA06B6823F040036B60194BAB604FF4166086
S3150C009CB0FFF7F2FE174BAB604FF46160FFF7ECFE5B
S3150C009CC0154BAB604FF49650FFF7E6FE134BAB60AB
S3150C009CD041F27070FFF7E0FE114BAB604FF4E150B0
S3150C009CE0FFF7DAFE6660FFF70BFF70BD004200500F
S3150C009CF00044005010470050004700506BCA5F6B81
S3150C009D00002F0B0100460050050001000300200146
S3150C009D10002F0501002F0301002F0201002F010166
S3150C009D20002F000110B54FF00053044C0FCB84E804
S3150C009D300F00FFF7BFFEFFF729FF10BDC4FF03207E
S3150C009D4008B501F0F9F908BD2DE9F04184B04FF4DE
S3150C009D5080330293002404AD05F80C4DDFF8D8804F
S3150C009D60404609212A4600F035F98DF80440304E5C
S3150C009D70304604212A4600F02DF98DF80440304671
S3150C009D8002212A4600F026F98DF8044030460321BC
S3150C009D902A4600F01FF98DF80C4088278DF80470C0
S3150C009DA0304605212A4600F015F98DF80C408DF841
S3150C009DB00470304608212A4600F00CF98DF80C4048
S3150C009DC08DF80470304609212A4600F003F98DF807
S3150C009DD00440404608212A4600F0FCF88DF80C4059
S3150C009DE08DF80470304607212A4600F0F3F88DF8FA
S3150C009DF00440304621462A4600F0ECF8304621460F
S3150C009E00012200F001FD4FF0806364F3010364F35B
S3150C009E108303022262F3092362F38B2364F38F33E9
S3150C009E20012262F39753034A136004B0BDE8F08134
S3150C009E300082024840400050008F024810B5234C67
S3150C009E40204600F0BBFB2268136823F480131360D2
S3150C009E5001F072F900F59C54083403E001F06CF93A
S3150C009E60A04205D21948002100F0A4FC0028F5D028
S3150C009E70164C20460021164A00F070FC2268136826
S3150C009E8043F490431360236841F21802995841F445
S3150C009E9000519950196841F00801196023689958C6
S3150C009EA041F0020199501A6842F004021A60094BFB
S3150C009EB008221A7000225A7027229A706922DA70C8
S3150C009EC05B221A7145225A7110BD00BF4088FE1FD5
S3150C009ED0F8B100087C88FE1F08230370002343702A
S3150C009EE0272383706923C3705B2303714523437156
S3150C009EF0704700BF10B5094800F0F8FA0446421E38
S3150C009F0040F2F3539A4205D804480549224600F01C
S3150C009F10BBFA00E00024204610BD00BF4088FE1F9F
S3150C009F20008AFE1F284B1B88013B9BB240F2F35262
S3150C009F30934248D8254B5A6993F826305B01D118C1
S3150C009F40D358002B0ADA214B1B68022141F214026A
S3150C009F509950002141F204029950704789680023F8
S3150C009F6003E01B4AD25CCA540133174A12889A4240
S3150C009F70F7D8164B596993F8260001EB40114A6045
S3150C009F8093F8262083F8282058695201815841F00D
S3150C009F900041815093F826200132D2B283F8262054
S3150C009FA093F825309A4203D10022084B83F82620D9
S3150C009FB0064B00221A621B68022041F2140158500B
S3150C009FC041F204015A507047B489FE1F4088FE1FA7
S3150C009FD0008AFE1FF0B48B081F1D50F8276001F095
S3150C009FE00305ED00F824AC4026EA040440F82740AB
S3150C009FF0466F4F000324BC4026EA04044467184C01
S3150C00A000A04203D004F58074A04207D1046E012649
S3150C00A01006FA01F124EA0101016617E054688C4046
S3150C00A0204460CC08103450F8247001F00701890004
S3150C00A03007268E4027EA060640F8246050F824705E
S3150C00A040167A06FA01F1394340F82410043350F815
S3150C00A05023101278AA400A4340F82320F0BC70471C
S3150C00A060008E0248030F20F0704003EB43039B0065
S3150C00A070014A9850704700BF14440050034B1868AF
S3150C00A080034B5B6903F00103D8407047C0FF032004
S3150C00A09000460050014B5860704700BF0046005008
S3150C00A0A0030F20F0704003EB43039B00014A9850CA
S3150C00A0B0704700BF484600502DE9F04142F2107E31
S3150C00A0C00027BC46012638E00B6803EB83035B00D4
S3150C00A0D0B3FBF6F34D68B3FBF5F4374AA2FB0482E7
S3150C00A0E0D20802EB82025200A21A052A05D9324A7C
S3150C00A0F0A2FB0442D208013203E02F4AA2FB04421F
S3150C00A100D2082AB102EB82046400B3FBF4F304E038
S3150C00A110294AA2FB0323DB080122AB4201D35B1BBA
S3150C00A12000E0EB1A142A07D89E4505D9B3F57A7FB9
S3150C00A13006D39E461746B4460136402EC4D901E0D6
S3150C00A1401746B44642F2107E0126402212E042F235
S3150C00A150107302FB0333B3FBF7F30C899C4201D853
S3150C00A1601D1B00E0E51AAE4501D9AE461646A342C4
S3150C00A17002D3013A022AEAD8BB1B026842F040021B
S3150C00A1800260023B1B0303F4E0434A89013A920145
S3150C00A190D2B21343721E120202F4706213430CF114
S3150C00A1A0FF3C0CF03F0C43EA0C030361036823F0FD
S3150C00A1B040030360BDE8F081CDCCCCCCD0F8C431E3
S3150C00A1C013F4407FFAD10131120442F0020242EA42
S3150C00A1D00161C0F8C411704738B50446074D2846CE
S3150C00A1E0FFF75EFF2846FFF73DFF236823F00103C8
S3150C00A1F02360236813F0020FFBD138BD100000104A
S3150C00A200D0F8C83123F00F031943C0F8C8117047B2
S3150C00A210D0F8C80100F00F00704700BF08B5FFF773
S3150C00A220F7FF012802D0022803D005E0FFF726FF2E
S3150C00A23008BDFFF761FC08BD002008BDF8B5044653
S3150C00A2400E461546FFF7C8FF20463146FFF7D8FFE6
S3150C00A2502046FFF7E3FFB0FBF5F2C2F58062002A59
S3150C00A26038BF002240F2FF37BA4228BF3A46C2F541
S3150C00A2708061B0FBF1F1AE098009B602B6FBF0F3D2
S3150C00A280BB4228BF3B4603FB00F0800A691AA5EBCC
S3150C00A290801081428CBF0020012000B1134608B10A
S3150C00A2A0012100E00221E26822F4434222F0FF027F
S3150C00A2B0E260E26843EA81331343E360F8BD00BF12
S3150C00A2C0037E012B17D103682022DA6101680B6823
S3150C00A2D023F07062037B1B0603F0706313430B6061
S3150C00A2E0036802691A61036842695A610368034A82
S3150C00A2F0DA61002070470320704700BF4000280039
S3150C00A300026802F13843A3F5A833990AC3F3441340
S3150C00A3101B0243EA4133916821F47F419160026844
S3150C00A32091680B439360037E012B2FD810B50368FD
S3150C00A3302022DA61C37913F0200F0ED1426802F0A5
S3150C00A340604343EA824302689361826802F0604389
S3150C00A35043EA82430268D36005E0036842689A6167
S3150C00A36003688268DA600446037E012B06D1FFF788
S3150C00A370A7FF23684FF00062DA6103E003684FF42D
S3150C00A3800062DA612368024ADA6110BD704700BFC9
S3150C00A3904000A0060368D969DA69C2F3800211F499
S3150C00A3A0006F0FD182B91A6902615A694261D96983
S3150C00A3B0DA69C2F3C00211F0040F07D0002AF2D1F9
S3150C00A3C0002070470320704702207047002070471A
S3150C00A3D030B400221EE0016953014FF00044CC500A
S3150C00A3E00169194444F2F4544C60016919448569B5
S3150C00A3F040F2F45404FB02548C60013290F82410A1
S3150C00A400914201D0144600E0002401690B4401EB93
S3150C00A4104411D96090F824309342DCD80268016963
S3150C00A42041F20C03D150002380F8273030BC704722
S3150C00A43030B4002318E041695A01124C8C50416922
S3150C00A4401144C56940F2F45404FB03548C60013387
S3150C00A45090F82510994201D01C4600E00024416971
S3150C00A4600A4401EB4411D16090F825209A42E2D8B7
S3150C00A4700268416941F21003D150002380F826305E
S3150C00A48030BC70470000103038B5044615460369D9
S3150C00A49090F8270003EB40130846996800F090FEED
S3150C00A4A0226994F827305B014FF00041D15094F8A3
S3150C00A4B027300133DBB284F8273094F824209342FA
S3150C00A4C002D1002384F82730236841F214029A58EB
S3150C00A4D012F0800F08D0802141F2140299502268A4
S3150C00A4E0002141F20803D150284638BD026990F884
S3150C00A4F027305B01D058002808DB00F40343B3F582
S3150C00A500407F05D1C0F30D400438704700207047DA
S3150C00A5104FF0FF30704700BF194B1B68194A126980
S3150C00A52002F0010293405B080168174A934203D874
S3150C00A53008230B6100207047144A934203D80C235E
S3150C00A5400B6100207047124A934202D80020086122
S3150C00A5507047104A934203D804230B6100207047BE
S3150C00A5600D4A934203D810230B61002070470B4A07
S3150C00A570934203D814230B610020704702207047C6
S3150C00A580C0FF032000460050C00E1602008793033E
S3150C00A59000E1F50580D1F00800C2EB0B80B2E60EA7
S3150C00A5A010B50420FFF776FD034C2046FFF778FD27
S3150C00A5B02046FFF757FD10BD0400002038B50446B1
S3150C00A5C0FFF7EEFF236803F580531A6842F0010289
S3150C00A5D01A60236803F580531B6813F0010FF8D13A
S3150C00A5E02046FFF799FF0546A268E16823681964BF
S3150C00A5F023685A6423684FF480621A6023688022A9
S3150C00A6009A612268144941F21803D150236803F564
S3150C00A6108053124A1A602046FFF7DAFE2046FFF7EF
S3150C00A62007FF22684FF0FF3141F21403D150226824
S3150C00A6306FF07C43C2F810312268C2F80C312368E3
S3150C00A6406FF0C022C3F8002223684FF40272DA635B
S3150C00A65000232362284638BD040020028020010214
S3150C00A66030B405682C6904F03C0444EAC12141EA83
S3150C00A670821242F001022A61002201680C6914F070
S3150C00A680010F03D14A691A80002005E001324FF60A
S3150C00A690FE718A42F1D9022030BC704710B40468AE
S3150C00A6A063610468236903F03C0343EAC12141EA70
S3150C00A6B0821242F00303236100230268126912F02E
S3150C00A6C0010F06D001334FF6FE729342F5D90220E4
S3150C00A6D000E000205DF8044B704700BF30B583B036
S3150C00A6E005460C4602220DF10603FFF7B9FFA0B989
S3150C00A6F028462146032201ABFFF7B2FF78B9BDF815
S3150C00A7000630222B0DD1BDF8043023F00F039BB27B
S3150C00A710B3F5AB5F07D0032006E0042004E0042069
S3150C00A72002E0032000E0002003B030BD30B583B05A
S3150C00A73005460C4600224FF40043FFF7AFFF0346D5
S3150C00A74053B92846214600220DF10603FFF788FF70
S3150C00A750BDF90630002BF4DB03B030BD70B50646F0
S3150C00A7600D461446FFF7BAFF034608BB304629468A
S3150C00A770FFF7DCFF0346D8B96388B3F5804F01D0E9
S3150C00A780002301E04FF40053A288B2F5006F01D10B
S3150C00A79043F48073A2790AB143F48053E2790AB187
S3150C00A7A043F48043304629460022FFF777FF0346E1
S3150C00A7B0184670BD00B583B001220DF10603FFF7F4
S3150C00A7C04FFFBDF8063003F004039BB20BB101201A
S3150C00A7D000E0002003B05DF804FB00BF30B48B082A
S3150C00A7E0043350F8235001F00301C900F8248C40BF
S3150C00A7F025EA040440F8234050F823408A402243BB
S3150C00A80040F8232030BC704710B4436F4900032432
S3150C00A8108C4023EA04034367436F8A401A4342671A
S3150C00A8205DF8044B704700BF70B505460E4600F048
S3150C00A830E3F8F47904B9102428463168224600F06E
S3150C00A84035F8B379013B64080134240244EA430326
S3150C00A85043F4403343F00103EB633379013B1B06AE
S3150C00A86043F481736B6373792BB16A6B013B42EAD8
S3150C00A87003436B6305E06A6B3379013B42EA03439E
S3150C00A8806B634FF4A063AB634FF0FF33EB64338918
S3150C00A8902B6470BDD0F80C3113F0E06F02D1406D13
S3150C00A8A080B27047D0F81C0180B2704763293BD93F
S3150C00A8B0002A3BD02DE9F04115460C460646FFF71B
S3150C00A8C0DDFB1B49A1FB00377F09A1FB04314809BD
S3150C00A8D040F2FF3E4FF0010CE046714611E001FBE1
S3150C00A8E007F305FB00F2B3FBF2F39C0AC3F309036F
S3150C00A8F0B4F5806F04D2734502D29E46A4468846B0
S3150C00A90001390029EBD148F4004333617269094BD4
S3150C00A9101340013D43EA85230CF1FF3C43EA0C430B
S3150C00A92073610020BDE8F08101207047012070475B
S3150C00A9301F85EB51EF8000FC30B4D0F8084124F0B1
S3150C00A940E064C0F80841D0F80851064C2C4041EAA6
S3150C00A950032343EA026244EA0203C0F8083130BC1E
S3150C00A960704700BFC0C0FFF830B4D0F80C4124F0DB
S3150C00A970E064C0F80C41D0F80C51074C2C4041EA6D
S3150C00A980032343EA026244EA020343F08053C0F80D
S3150C00A9900C3130BC704700BFC0C0FFEF10B5114B77
S3150C00A9A0984208D14FF40060FFF77AFB4FF4006031
S3150C00A9B0FFF758FB10BD0C4B984207D10B4C2046A9
S3150C00A9C0FFF76EFB2046FFF74DFB10BD084B984278
S3150C00A9D006D1084C2046FFF763FB2046FFF742FBE7
S3150C00A9E010BD00BF0800034008000248800000109C
S3150C00A9F0084002480001001010B50446154B984259
S3150C00AA0003D003F50073984203D11348FFF7C6FF32
S3150C00AA1014E0124B984203D003F50073984203D10D
S3150C00AA200F48FFF7BBFF09E00E4B984203D003F526
S3150C00AA300073984202D10C48FFF7B0FF0323E36082
S3150C00AA40E36813F0010FFBD0236C23F00F03236490
S3150C00AA5010BD00BF00000340080003400000024880
S3150C00AA60080002480040024808400248704700BFF0
S3150C00AA702DE9F0438BB04FF46143019308238DF815
S3150C00AA8008308DF8093001258DF80A5010278DF8FD
S3150C00AA900B700026ADF80C601C4C204601A9FFF784
S3150C00AAA0C3FE8DF81C6008954FF002098DF82490B2
S3150C00AAB0DFF85C804046042107AAFFF78BFA902347
S3150C00AAC08DF8103005958DF81890404605210DEB44
S3150C00AAD00702FFF77FFAE36923F007032B43E361D1
S3150C00AAE02046394604222B46FFF726FF20463146E0
S3150C00AAF004222B46FFF738FF236C23F00F0343EA9F
S3150C00AB00090323640BB0BDE8F08300BF00000340CB
S3150C00AB100081024830B58BB0FFF7B0FA044600E06E
S3150C00AB206400434B9C42FBD900E06408414B9C42B9
S3150C00AB30FBD8414801212246FFF780FB01943F4B8D
S3150C00AB4002934FF4FA53ADF80C300123ADF80E30E6
S3150C00AB503B4C204601A9FFF7AFFA236843F04003AC
S3150C00AB602360236843F001032360364B3648186094
S3150C00AB70DA79022161F38712DA71596840F2676457
S3150C00AB8064F31C0159609A6864F31C029A60090EFE
S3150C00AB906FF34511D971120E42F02002DA72C268B7
S3150C00ABA042F00052C26008221A73002305E0254ABF
S3150C00ABB01A44002111740133DBB2072BF7D9214853
S3150C00ABC000250576FFF79CFB1B4801210A46FFF77B
S3150C00ABD0F5FA1B4C236823F040032360236823F00B
S3150C00ABE0010323600AAA02F80C5D184D28460D21B4
S3150C00ABF0FFF7F0F990238DF810300123059302230B
S3150C00AC008DF8183028460C2104AAFFF7E3F92368BF
S3150C00AC1043F040032360E36823F0070343F0020389
S3150C00AC20E360236823F0400323600BB030BD00BF04
S3150C00AC30FF1AB700000E27070040014820A10700A5
S3150C00AC40004301487889FE1F2050014800810248C4
S3150C00AC50074BD3F8143113F0080F07D110B504467F
S3150C00AC600348FFF717FE2070012010BD0020704727
S3150C00AC700000034008B5FFF7FBFEFFF74BFF08BDCE
S3150C00AC80BFF34F8F0549CA6802F4E062044B1343C5
S3150C00AC90CB60BFF34F8F00BFFDE700BF00ED00E0B8
S3150C00ACA00400FA0508B5204B1B78ABB91F48FFF713
S3150C00ACB0CFFF012837D11D4B1B78013BDBB23F2B55
S3150C00ACC031D800F039FA1A4B18600122164B1A705B
S3150C00ACD00022184B1A7008BD164B1B7816481844E0
S3150C00ACE0FFF7B6FF012814D1124A13780133DBB2F1
S3150C00ACF013700E4A1278934215D100220A4B1A7021
S3150C00AD000A4B5B78FF2B0ED1084B9B785BB9FFF790
S3150C00AD10B7FF00F011FA064B1B686433984202D950
S3150C00AD200022014B1A7008BD6C89FE1F2889FE1F74
S3150C00AD307089FE1F2489FE1F2989FE1F00B583B06A
S3150C00AD40174B1B68DB6913F0010F1BD01448FFF778
S3150C00AD5021FB60B1002210E0114A1A44117C02AAB0
S3150C00AD601A4402F8081C0133DBB2012201E000226E
S3150C00AD7013460B49097B9942EED8094B1B680121F6
S3150C00AD80D96100E0002242B19DF80030FF2B04D1BE
S3150C00AD909DF801300BB9FFF773FF03B05DF804FBA8
S3150C00ADA07889FE1F08B5FFF77DFFFFF7C7FF08BDC3
S3150C00ADB010B5054C204608218022FFF70FFD4FF0F9
S3150C00ADC08073636010BD00BF0085024808B500F0B3
S3150C00ADD0B3F90D4B1B68C31AB3F5FA7F13D30B4BA0
S3150C00ADE01B783BB90122094B1A704FF48072084B41
S3150C00ADF05A6006E00022054B1A704FF08072044B25
S3150C00AE005A60014B186008BD9889FE1F9C89FE1F6D
S3150C00AE100085024808B5FEF773FEFFF7C9FF00F080
S3150C00AE2069F908BD08B5FFF7F5FF00F02FF900F03A
S3150C00AE300DF8FFF71FFF0020014600F03FF9FFF762
S3150C00AE40C5FF00F059F8FFF7ADFFF8E710B5FEF7B0
S3150C00AE507BFF00F071F900F5FA70134B186000F0E7
S3150C00AE606BF900F51C501030104B1860FDF77AFA90
S3150C00AE700F4A0023138053800E4A138053800E4AC8
S3150C00AE80138053804EF60300FDF7ACFAFEF7D6FF9F
S3150C00AE900A4C2046FFF720F820460621FEF78EFCCA
S3150C00AEA0FEF7AAFC10BD00BFAC89FE1FA089FE1FD1
S3150C00AEB0FC89FE1FF889FE1FF489FE1FA489FE1F5C
S3150C00AEC008B50B4B1B7813F0400F0FD113F0020F84
S3150C00AED00CD0084B1B681A79FF2A07D15B792BB962
S3150C00AEE00020012100F0EAF8FFF7CAFE08BD00BFFA
S3150C00AEF0C089FE1FC889FE1F10B5FEF7FBFF48B3BD
S3150C00AF00384A1080384B9C894FF40060FDF784FA60
S3150C00AF1084420DD10120FDF7B9FA324B1B88CBB117
S3150C00AF20FEF754FAFEF7FEFF00222E4B1A8011E0B4
S3150C00AF302D4B9C8940F60600FDF76EFA844209D12A
S3150C00AF40FEF7CEF9274B1B8823B1FEF7EBFF002249
S3150C00AF50244B1A8000F0F0F8244B1B68984233D32C
S3150C00AF6003F5FA73214A1360002414E0C4EB0412AF
S3150C00AF7052001F4B13441F4A13600220FDF786FA3A
S3150C00AF80184B1B8833B1FEF721FAFEF7CBFF0022D4
S3150C00AF90144B1A800134002CE8D0002412E0164B16
S3150C00AFA003EB8413154A13600520FDF76FFA0D4B5E
S3150C00AFB01B8833B1FEF70AFAFEF7B4FF0022094BE1
S3150C00AFC01A800134002CEAD000F0B6F80C4B1B6842
S3150C00AFD0984206D303F51C531033094A1360FEF747
S3150C00AFE047F910BDB489FE1F008AFE1FAC89FE1FEF
S3150C00AFF0D089FE1FCC89FE1F4490FE1FC489FE1FFC
S3150C00B000A089FE1F0C4B1968C1F3072353FA81F371
S3150C00B010C1F307421A440B0E13FA82F39BB20022B9
S3150C00B02005E005491144087903449BB20132372ADD
S3150C00B030F7D9584280B270470080FE1F08B5FFF75B
S3150C00B040E1FF044B9B8F984201D0002008BD0120E4
S3150C00B05008BD00BF0080FE1F08B5064B1A68064BDC
S3150C00B0609A4203D1FFF7EAFF10B908BD002008BDCC
S3150C00B070012008BD0080FE1FA2E742CE08B5FFF7EF
S3150C00B080C1FF014B988708BD0080FE1F08B5FFF76E
S3150C00B090E3FF68B9074A084B1A60002304E0064A26
S3150C00B0A01A44002111710133372BF8D9FFF7E6FF4B
S3150C00B0B008BD00BFA2E742CE0080FE1F38B504468D
S3150C00B0C00D46FFF7C9FF40B1372C08D8054B1C4479
S3150C00B0D02571FFF7D3FF012038BD002038BD0020B5
S3150C00B0E038BD00BF0080FE1F014B1860704700BFC3
S3150C00B0F0B089FE1F08B50C4B1B680C4AA2FB032338
S3150C00B1009B09013BB3F1807F09D2094A5360FC21AC
S3150C00B110084B83F823100023936007231360002049
S3150C00B120FFF7E2FF08BD00BFC0FF0320D34D62103E
S3150C00B13010E000E000ED00E0014B1868704700BF1E
S3150C00B140B089FE1F024A136801331360704700BFB3
S3150C00B150B089FE1F70B50E4B0E4CE41AA4100025D8
S3150C00B1601E46A54204D056F8253098470135F8E717
S3150C00B170FFF77CFC084C094BE41AA41000251E466C
S3150C00B180A54204D056F8253098470135F8E770BD2E
S3150C00B1907088FE1F7088FE1F7088FE1F7088FE1F49
S3150C00B1A010B50A44441E914208D014F8013F0878A1
S3150C00B1B0834201D0181A10BD0131F4E7002010BDEE
S3150C00B1C010B5431E0A44914204D011F8014B03F802
S3150C00B1D0014FF8E710BD02440346934202D003F830
S3150C00B1E0011BFAE770470000FFFFFFFFFFFF00009F
S3150C00B1F0ADDE122363825363010000400008000099
S3150C00B20000C0005000000000080027695B450000E4
S3150C00B21020300020A02F0020D01700200000002096
S3150C00B2200000000004040000000000000000000004
S705080082056B
